:020000040000FA
:10000000CE0026BD28E2DE0FFF0808DE11FF080A39
:10001000F60110C4BFF70110D617C40FCE4027BD9C
:100020004C38B70102200401020408BD43A496170E
:100030004848F60103C4F31BB701039617D61811FD
:1000400026037E4091CEFFFFFF00D54D2B085D2A91
:1000500020BD600220065D2B18BD5FDB7D064527B5
:10006000037E40FEB606448AC0B70644C6807E4181
:100070000458581B840F16CE4082BD4C38164F7E54
:100080004104011419280A0114230F0A010F140F47
:10009000087D00172B3FCE00D5DFC5860297C79697
:1000A00026B105832514221E9625B10582250B2233
:1000B000157F00D57F00D67E40FECE0582DFC1CE03
:1000C0000025DFC3200ACE0025DFC1CE0582DFC3B5
:1000D000BD49AF20299626262596258112241F7D0D
:1000E000001E260CC604911D24149B25195A26F6C1
:1000F000BD5F9B860A5FCE41A7BD22C52063C600B7
:1001000086052010363786109A869786B70812BD66
:100110005F9B3332CE41AABD22C596FB2A43851090
:10012000260C85202624D6D6270BC103251CC68085
:10013000F701092015F60816C5102708D6D5C10500
:1001400025132006D6D5C102250B8A2084FB97FBF8
:10015000BD5CC9200CB60112840381032603BD5E79
:100160006BDE1FDF1BDE21DF1DBD6089D681270608
:10017000C1802702201D9645810126119680270DFA
:1001800086809181270D9781BD471F20067F0081C2
:10019000BD471FF601D3CA40F701D3F60106C501DA
:1001A0002703BD53184F39BD5F8BBD27C42617B633
:1001B000010185082610F60644C5012609860A5F56
:1001C000CE41AA7E22C57D00172B217D00182B1C55
:1001D000F60644C502271596FB2A068A2084FB975B
:1001E000FBBD5F9BC632CE41EC7E22C5BD5F8BB6A8
:1001F000064484FCB706447F00D7C6649645810157
:10020000261596468105240F96109014240143C6A6
:100210000181502502C614D7D8DE0FDF13DE11DFAF
:1002200015968684EF9786B7081286055FCE42330F
:100230007E22C5BD522E96998503271DD6FB2A081E
:10024000C5302704850127117A00D827177F00D7EA
:1002500086055FCE42337E22C596D74C81032404A7
:1002600097D720EC9617971896FB84FD97FBBD5403
:1002700000BD5E6BBD5CCEF601D3C4BFF701D3B643
:100280000C0B8A08B70C0BBD522EBD34E07F0085E5
:1002900096DB270DD6DC2709867D5FCE42947E2231
:1002A000C5BD5042BD5F8296452601392B1F810195
:1002B00027059683260139BD433E964681012203D8
:1002C0007E4EA7C6028671CE4EA77E22C5BD433E96
:1002D000964581822603BD319239FF012608080820
:1002E0004FAB0019A100264909BC012626F2E603FE
:1002F0002B37F1061F25372618E602F1061E252E9C
:10030000E601F1061D2527E600F1061C25207E43A7
:100310002CF1062325162611E602F10622250D26CC
:10032000086D0126046D0027038602394F398601C6
:100330003986583996868A019786B7081239968683
:1003400084F69786B7081239DEF2DF1FDEF4DF216C
:1003500036961897173239DE1FDFF2DE21DFF439C7
:10036000DE23DFF2DE25DFF4DE02DF23DE04DF251D
:10037000BD3D67DE23DF02DE25DF04DEF2DF23DEA4
:10038000F4DF259618971739B601018A80B7010165
:100390002024B601018A80B701012037B60101840B
:1003A0007FB701017D01012B29B60816850226239E
:1003B000D626C116251DB601018501271584FEB775
:1003C00001017D06452608B606448AC2B706447E6A
:1003D000547839B60101850126F88A0120E17F00B1
:1003E0008A20067F008A7C008ABD39329645271A0A
:1003F0002A158182260EB60137B10136270984FEFF
:10040000817027037E4F607F0044962E2619962D1B
:100410002615962C2611962B81042A0B4A91172A11
:10042000067F00897C0089BD4357CE0027DFC1CEFF
:10043000002BDFC3CE001FDFC5860497C7D68A27EF
:100440000FBD49AFBD3D568100271C86017E445932
:10045000BD4992BD3D564D270EF60116C50826032F
:100460007E52D54F7E52D59689260ADE1FDF27DEC3
:1004700021DF292008DE23DF27DE25DF2996658A94
:10048000829765BD34D29645270CBD434886819737
:1004900084BD64CD2003BD3FA6B60C08B10136264D
:1004A00020D68B270B7A008BC67ACE44997E22B059
:1004B0008604978BB60136814226037E43DE7E4357
:1004C000E38620978B7F008A7F0089B60C088142E3
:1004D00027058143270139B701367E4499B60114B7
:1004E0008880858027048A40200284BFB7011439A0
:1004F0007F01367E43DE7F01367E43E3B6011484FE
:100500003FB7011439B601148AC0B7011439CE08B7
:1005100005FF012CC60BD7967F00907F0095F60152
:1005200015F70091CA03D79BBD4988F60115CA0388
:10053000F70115D79BCECCCCFF0800FF0802FF08BF
:100540000439978EBD4988BD4977F60115F70091AA
:10055000D69BF70115FE012CC601D795D69626022B
:100560002023D690275ED6932706C1022702264075
:10057000968EBD45F1C60CD78D9A8DA700979C7AB3
:1005800000967F0090F60115D79BF60091F70115B4
:100590003902F60115C4FCCA02F70115969C8A0CB3
:1005A000A700C602D793D696F70092FF012E20D55A
:1005B00002F60115C4FCCA01F7011586008ACCA712
:1005C000007E45A2D6932704C10226C5968ED69CEE
:1005D000C4F0D78D9A8DA7007A009609FF012C7C74
:1005E0000090C6CCD78DF60115CA23F701157E45BC
:1005F000850C4949494939BD4988BD4977F60115F6
:10060000F70091D69BCA03F70115FE012CF60125D0
:10061000C58026037E465257251DB60140F60125AA
:10062000C47F1081012E0108BC012E2625F601157C
:10063000C4FEF70115201BBC012E260AF60115C4C5
:10064000FDF70115200CD690270808BC012E2602C4
:1006500020EA7C0096D690271C7F0090FE012C0893
:10066000FF012CFE012808E600BD4965FE012CCAE9
:100670000FE700200AFE012C7C0090C6CCE700D7D3
:100680009CF60115D79BF60091F7011539BD4988F5
:10069000BD4977F60115F70091D69BCA03F70115FE
:1006A0007F0093CE0000FF012EFE012CF60125579E
:1006B00025037E466302C6CCE7007E467FBD4943E4
:1006C000B60097B7080239860120308602202C86B2
:1006D00003202886042024860520208606201C86E8
:1006E0000720188608201486092010860A200C8608
:1006F0000B2008860C2004860D2000F60C08F10162
:100700003626159781BD471FC6FFCE47107E22B003
:10071000B60136B10C0827F07F0081BD471F39F6BE
:1007200001252716D69A2612F60116C5802601390C
:100730009681810E270139BD3932BD497796812ACC
:10074000037E485B8106260CCE0072BD47A4CE0016
:10075000767E47F2810726037E483F810826037E86
:1007600048D7810E26037E46BD810F26037E4902AF
:10077000811026037E49262B0586557E52D51658B4
:10078000CE4788BD4C24201C00230027002B0610D8
:1007900006140618003B006000DD0047004B004FC8
:1007A00000530057BD4943A603272785F026028A38
:1007B000F0B70803A602B70802F60115C4FEF70158
:1007C00015A601B70801CA03F70115A600B708006E
:1007D000200CA60227E385F026DC8AF020D896813B
:1007E0008105260A7D0082270586FDB7080439BDEC
:1007F0004943A60185F0260E81002629A60085F032
:10080000262CB7080539BD4960B70805E601BD4982
:1008100065A600BD49601BB70804E600BD4965CA6E
:100820000FF7080339B70805A600B7080439BD4912
:1008300060B70805E600BD4965CA0FF7080439BD71
:1008400049439661270B8AF0B708039660B7080200
:1008500039966085F026F68AF020F2BD4943B60647
:1008600013271485F02708BD49608AF0B70805F6FC
:100870000613BD49652009C6F0B6061285F0270AA1
:10088000B60612BD49601BB70804F60612BD4965DD
:10089000B60611BD49601BB70803B60617271485B5
:1008A000F02708BD49608AF0B70802F60617BD496F
:1008B000652009C6F0B6061685F0270AB60616BDED
:1008C00049601BB70801F60616BD4965B60615BD99
:1008D00049601BB7080039BD494396DD2723CE0880
:1008E0000496DE8D0E96DF8D0A96E08D0696E18DDC
:1008F0000296E22A0C5F5C44250220FACAF0E70067
:100900000939BD4943B6016016840F8B0019C4F044
:10091000270A575757578B16195A26FA85F0260279
:100920008AF0B7080239BD4943BD27C42708FE6ACB
:100930001CFF0802200CFE6A1CFF0803FE0648FF8D
:10094000080039F60115CA03F7011586FFB7080537
:10095000B70804B70803B70802B70801B708003999
:100960004444444439585858583986FFB701422006
:10097000D27F01427E471FB60817850427067D01F6
:1009800042260139313120BBF60116C50826023155
:1009900031390CDEC1A60008DFC1DEC3A900190889
:1009A000DFC3DEC5A70008DFC57A00C726E5399694
:1009B000C74A9BC2B700C996C18900B700C896C78D
:1009C0004A9BC4B700CB96C38900B700CAFE00C8D3
:1009D000E60009FF00C8FE00CAA60009FF00CA1110
:1009E000251B2607089CC3271420E2DEC1FF00C890
:1009F000DEC3DFC1FE00C8DFC3C68020015F0D86F5
:100A000000DEC38999A00008DFC3DEC1A900190870
:100A1000DFC1DEC5A70008DFC57A00C726E109EA05
:100A200000E70039CE0000DFAEDFB0DFB2DFA9DFC4
:100A3000ABDFACDFC1DFC6860197C57F00C3CE0048
:100A400006A69C26040926F939CE0006A6A2260988
:100A50000926F98666BD52D5397F00C396A2261FA6
:100A600096A8261B7C00C3CE000502A69CA79DA6C7
:100A7000A2A7A30926F57F009D7F00A37E4A5C5FA5
:100A80000202CE0000A69D260EA6A3260A085C8CB4
:100A9000000626F17E4A53F700C27F00C396A826BF
:100AA0001ABD4B397C00C396A82610BD4B397C007B
:100AB000C396A82606BD4B397C00C396A291A825F3
:100AC00002220FB600C32604BD4B6F397A00C3BDA6
:100AD0004B47CE0005DFAEA69DA1A32532270CDF34
:100AE000AEBD4B58BD4B6FDEAE20ECDFAE810027B4
:100AF00013A69CA1A2250926030926F5DEAE20DF58
:100B0000DEAE200BDEAE09260139DFAE7E4AD7B657
:100B100000C32601397A00C3DFAE96AD270586995A
:100B200097AD39BD4B86BD4B47CE0006A6A2260425
:100B30000926F939DEAE7E4AD7CE0005A6A2A7A3C4
:100B40000926F97F00A339CE0000A6A4A7A3088C2C
:100B5000000526F67F00A839FE00C10D86008999A0
:100B6000A0A3A99D19A79D088C000626EF39020CA9
:100B700096AA99C51997AA96AB99C61997AB96AC40
:100B800099C71997AC3996AC97AD96AB97AC96AA26
:100B900097AB7F00AA39B700C1F700C24444444470
:100BA000C60ABD4BE1B600C1840F1BF600C2BD4CA6
:100BB00018F700C1C60ABD4BE1FB00C18900B700B0
:100BC000C1860ABD4BE1F70006B70007B600C1C6F3
:100BD0000ABD4BE117F600C2C40FFB0006B90007BF
:100BE00039B700C37F00C47F00C57F00C6CE0008B0
:100BF00009542412B600C5BB00C3B700C5B600C671
:100C0000B900C4B700C67800C37900C48C000026C0
:100C1000DFB600C6F600C5395454545439098C0067
:100C20000026FA39FF0126FB0127F7012724037C60
:100C30000126FE0126EE0039FF0126FB0127F70100
:100C40002724037C0126FE0126A600396F011684A5
:100C50000F8B0019C4F0270B8B161924026C01C0EE
:100C60001026F5A70039968684FBB708129786965A
:100C70004585022703BD52248600974597839784B4
:100C80009785977B977C977DB601138A70B7011380
:100C9000BD4D97DE27DF1FDE29DF21BD3D4CBD5E48
:100CA0006B8658BD28E139964581112607B6064462
:100CB0008540270839D645C101260139B606448446
:100CC0007FB70644C1112607860197457E4EA78649
:100CD000019745B601138A7084EFB701138657BD9B
:100CE00028E15D26037E4DA22A1C968291F02716EC
:100CF00097F0BD51A896F1270DBD51A8BD4348DE20
:100D0000F6DF7C7F00F18602C671CE4EA77E22C53B
:100D1000D645260486019783D645378602974586B1
:100D200057BD28E1B601138A7084BFB70113335D44
:100D300027707E4DBB968684FBB708129786D645F2
:100D4000C1022603BD522486809745B601138A70DE
:100D500084DFB701135D274A7F0081BD471F865896
:100D6000BD28E139867FB7013720A58668B70137EE
:100D70007F008320A386FF97DB39D645868297457F
:100D80008657BD28E1BD4D97B601138A70849FB781
:100D900001135D270D202496DB2601397F00DB7EC1
:100DA0003031F601EA2703BD4D757D00652A0CBD83
:100DB000672E9665847F97657E6638B60644847F85
:100DC000B706448602B70645964584EF9745968652
:100DD00084FBB708129786964581022603BD5224EC
:100DE000CE0000DF7CFF05797F0084BD5E6B7D0651
:100DF000442A0F9645810126098A10974586167E5A
:100E000052D5D6DB2703BD30E0DE66DF1FDE68DFAC
:100E100021BD3D4C4D272D9682260CFE061CDF1F62
:100E2000FE061EDF21200AFE0620DF1FFE0622DF4F
:100E300021BD3D4CDE66DF1FDE68DF21F60110CAF2
:100E400040F70110BD5042D665C5022709D665C4DA
:100E500040D765BD623EBD513CD682D7F096452A4B
:100E6000058601978339D645C1022613B60137811D
:100E700068270481762604968327047F00833996A9
:100E8000868A04B708129786C1022605BD5224201F
:100E90000DB601138A10B7011384EFB70113860151
:100EA000978396469787397D0639270AB6081785AE
:100EB00008260DBD4334C6028671CE4EA77E22C5DC
:100EC000BD433E9687270D7A0087C6048642CE4EE4
:100ED000C37E22C596464A9787D6F1270C7F00F13C
:100EE000BD4348DEF6DF7C204996822615BD505F63
:100EF000BD50FBBD50874D261E96DB2735BD30F714
:100F00002030BD5073BD50FBBD50B54D260996DB5A
:100F10002720BD3109201B968684FBB708129786CF
:100F2000BD34D6D645C1022603BD52247C00857E41
:100F30004DE0BD5156BD3D4C81002715C60286715E
:100F4000CE4EA7BD22C5BD5042F60110CA40F701E2
:100F500010D6F1C402968684FD1B9786B708123915
:100F600096DB270796DC27037E4499D6DD27487F4A
:100F700000EED68AD1F027217A00EED7F0968A9833
:100F800082270CBD520FD6F1272DBD520F200ABD6E
:100F900051A8D6F12721BD51A8D6F1271A7F00F11B
:100FA000BD4348DEF6DF7C968A98822606D6EE267A
:100FB000062053D6EE2757D68A2621BD505FD6820B
:100FC0002605BD50872003BD509E4D2609D6DB2740
:100FD0002CBD30F72027BD50737E5033BD5073D6E3
:100FE000822605BD50D82003BD50B54D2609D6DB5D
:100FF000270BBD31092006BD505F7E5033968A987D
:10100000822608BD50FBBD51562006BD5110BD5172
:10101000BDBD3D4C4D270BBD5042F60110CA40F7F7
:101020000110D6F1C402968684FD1B9786B708127C
:101030007E44999645818226037E3192BD34D67EC8
:1010400044C1DE7CFF0810FF057939B60579800AB6
:101050002409F6057A5A2B06F70811B7081039CE7D
:10106000001FDFC1DFC5CE0072DFC3860497C7BD96
:10107000499239CE001FDFC1DFC5CE0072DFC386C3
:101080000497C7BD49FD394FD6222B11CE0004E687
:1010900069E11E220825050926F520014C394FD6A5
:1010A000222B11CE0004E665E11E22082505092643
:1010B000F520014C394FD622C1502406D66D2B178E
:1010C0002004D66D2A10CE0004E61EE16922082510
:1010D000050926F520014C394FD622C1502406D6E9
:1010E000692B172004D6692A10CE0004E61EE1659C
:1010F000220825050926F520014C390C96789B7BA2
:1011000019977B9679997C977C967A997D977D390A
:10111000967C9079977C967D927A977D9678271B1E
:101120000D860089999078997B19977B250D0C96EF
:101130007C8001977C967D8200977D39CE00DEFF12
:101140000130CE00E3FF0132860097F1968684FDE0
:101150009786B7081239D6DD2762FE01308C00E38E
:10116000275AE6002B05BD51A820EFFE0132E6010B
:10117000D17D250A2646E600D17C2502263EBD43C8
:1011800057DE7CDFF6FE0132EE00DF7CFE0130A68A
:1011900000BD6381A600971FA6019720A602972194
:1011A000A603972286FF97F1FE01308C00E3270CFF
:1011B00008FF0130FE01320808FF013239D6DD2771
:1011C00062FE01308C00DD275AE6002B05BD520F70
:1011D00020EFFE0132E601D17D220A2646E600D14B
:1011E0007C2202263EBD4357DE7CDFF6FE0132EE56
:1011F00000DF7CFE0130A600BD6381A600971FA61C
:10120000019720A6029721A603972286FF97F1FE59
:1012100001308C00DD270C09FF0130FE0132090985
:10122000FF013239CE2C66BD4C1D392001EFB60CC2
:101230000BB60C0A840F9799B7064748484848B739
:101240000C0A44444444F60C0AC40F1126E0D61795
:101250002A19B6064784FDF60646C4021B979985EF
:10126000012608F60646C4011B97997D01D3271471
:10127000F60110C4F784081BB7011096998AF8B4D8
:1012800001102008F60110C4F096991BB701107EDA
:1012900034EBB606268403B70646D6172BA839B614
:1012A0000C08B10136261F860E9781BD471FC6FF69
:1012B000CE52B67E22B0B60C08B10136260220EE20
:1012C0007F0081BD471F4F200C9697811627F18123
:1012D000202BF3203D4D270A7D00972A0591972466
:1012E00001399797260AF60114CA30F70114202213
:1012F000F60114C4EFF701148116270C81202B127C
:1013000026067F00437F0088F60114C4DFCA10F769
:101310000114BD34AD969739F601D3CA20F701D335
:10132000C614F701EB200B96998507270D7A01EB80
:101330002716C6FFCE53277E22D5C618CE53427E2F
:1013400022D59699850726DFF601D3C4DFF701D3AE
:10135000BD522E7E34E0D643C11125048653202B86
:10136000C106260ED69AC10626048607201D8605CC
:101370002019CE538EFF0126FB0127F701272403F6
:101380007C0126FE0126A600B700987E52D52101D9
:10139000020101010708090101010101242424BD02
:1013A0005413B60111850826092024B601118508B9
:1013B000261D96FB841E97FB7F00FCF60111CA08D0
:1013C000F701117F010B7F010CBD59297E58F77F72
:1013D00000FC96FB8501271184FA97FB8680B701F4
:1013E00009C618CE53CF7E22D58A8097FBF601110D
:1013F000C4F7F701117E545C7F00FC7A00FC20D218
:1014000096FB2A04853026083996FB2B037E592942
:101410007E54AB8680B701097F010B7F05827F0573
:101420008396FB85102703BD584239BD53B27E53C6
:101430009FBD5413BD53B2860197FB96FB271785BA
:10144000012713F60109C4FECB02F701095F867D6F
:10145000CE543B7E22D53996FB851039D6FB2A1710
:10146000C5082613CA20D7FBC512260B96452B04A8
:1014700085032603BD54AB39D6FB2A1BCA20D7FBF4
:10148000C502261396452A0F8503260BC662CE5445
:10149000947E22C5BD54AB3996FB85102708B60152
:1014A0000A850427013931317E54137D00172A0340
:1014B0007E5413D6FBC5102712C680F7010930EE03
:1014C000008C5477270D8C5497270832B7060E32BC
:1014D000B7060FBD5CC9D617C1022507F60101C5C5
:1014E0000126058608BD6062B6010384FD8A01B746
:1014F0000103B6010684FDB70106F60104C4FBF73B
:101500000104B6010A8502260CB60105850C2605E4
:101510008604B70105F601D3CA80F701D396FB858F
:101520000427037E5705CE0001B601168508260460
:1015300096FC262096D6260BD6FBC5102716CE0481
:101540007020112B0CCE06A881032508CE16312061
:1015500003CE2C64964581012703BD4C1D7F00F806
:10156000D6FBCA10D7FBCE5570C60486E27E22C5D4
:10157000BD5498BD522E9699850527057C00F82606
:10158000E5B601048A08B70104DE25FF0582BD59CE
:1015900029B6064485042740B60101850826397F0F
:1015A00006388659BD28E17D0639262C7D06382A65
:1015B000F6C69CBD590DBD5918BD58D7BD58EEB6DD
:1015C00008172B0F86FFBD29167D0639260A7D08D0
:1015D000172AF67D063927E7F60638C40FF70638CE
:1015E00027037E5842C69CBD590DBD59187F00F98E
:1015F0007F00FA7E569896F98102260586907E59DC
:10160000027C00F97F00FAC680F70109BD591EC6A9
:1016100018CE56177E22C5BD5498C69CBD590DBD27
:101620005918860297F8BD58E5BD58D7B60109800C
:1016300006810824037E55F6B70109CE000BBD4C88
:101640001DB608172A0A96F827037A00F87E56294D
:1016500096F8260BB601098B06B701097E568F86D0
:101660000297F8BD58D7B601098B0681F825037E8D
:1016700055F6B70109CE000BBD4C1DF608172BDF40
:1016800096F827067A00F87E5663B601098012B7ED
:101690000109CE00E4BD4C1DB6010981F025037E91
:1016A00055F6BD58D7BD58EEB6010997FD8B01B769
:1016B0000109CE000BBD4C1DF608172A0781F8253D
:1016C000EC7E55F6B6010997FE96FD8001B701093B
:1016D000CE000BBD4C1DF608172A07810824EC7EAE
:1016E00055F6B6010999FE46B7010990FD2A014356
:1016F000811425117D00FA260C7C00FACE00E4BD91
:101700004C1D7E5698BD58F7BD591ECE0017BD4CD6
:101710001D966226058608BD603CF6011253C5037E
:1017200026037E5842BD5E89B6010AB7060B8A01C0
:10173000B7010AF6010FF70609B60108B7060ABD98
:101740005F467D06072A37B70607B70608BD5F6004
:10175000BD57C8FE060CE600A641098C0584270685
:10176000E700A74120F4B60609BD600BF6060AF7AC
:101770000108B6060BB7010ABD5E6B7E5842B10682
:10178000072420F60607B7060717BD5F604A2BC37C
:10179000B1060725BEFE060C09FF060C36BD57C86C
:1017A0003220EAF6060811240220BBB7060817BD4E
:1017B0005F604CB10608270224ACFE060C08FF0649
:1017C0000C36BD57C83220EAF6010F484824048B76
:1017D0009E200AC508260C816025068062C4F72079
:1017E00008CA0881B024F48B02B7010817BD600B4A
:1017F000CE0017BD4C1DC602F700064FB7010B9A6D
:1018000006B7010C020202F60817C5102702980657
:1018100074000626EAB7010CFE060CA741C680F745
:1018200000064F9A06B7010B020202F60817C51010
:101830002702980674000626EAB7010BFE060CA7DD
:10184000003996FB84C08A0897FBBD591EBD5E6BAC
:10185000BD58EE966226058608BD603CBD5A40B66E
:1018600001124384FC27342A05BD5BD52030854016
:101870002705BD5BA6202785202705BD5B77201E99
:1018800085102705BD5B47201585082705BD5B181A
:10189000200C85042708BD5AE92003BD5ABCBD5C55
:1018A000CEB6011185102703BD5DEABD59C396FB75
:1018B00084C097FB7F00D6F601D3C47FF701D3BD68
:1018C000522EBD34E0FE060E27087F060E7F060F5F
:1018D0006E0086897E52D5B601048A08B701048459
:1018E000F7B7010439B6010484FEB7010439B60123
:1018F000048A01B7010439969781902701394F7EF8
:1019000052D5D6FB2A03BD52D5BD541339B60C0AA5
:10191000850227035A26F6398604BD603C398604C1
:10192000B5010F2703BD6062397D060C2601394FD2
:10193000CE0585A700088C060D26F8B7010BB70168
:101940000C4AB70607B7060839B601118AC0B701B5
:1019500011B601048A02B70104B6010684FDB7017D
:1019600006BD5E6B8643BD28E139B601118AC0848D
:10197000BFB701118644BD28E1BD545726187D002C
:10198000172B13B601048A02B70104B601068A02B6
:10199000B70106BD5E6B39B601118AC0847FB701FD
:1019A000118645BD28E1BD545726EB7D00172BE677
:1019B000B6010484FDB70104B601068A02B7010628
:1019C0007E5E6BB601112B05BD59A620078540260A
:1019D00003BD597939B601118A0684FEB701118613
:1019E00046BD28E17D00172B31B6010384FD8A0135
:1019F000B101032725B701037E5FA4B601118A0553
:101A000084FDB701118647BD28E1BD5457260BBDA3
:101A10005A5DB6010384FDB7010339B601118A038B
:101A200084FBB701118648BD28E1BD545726EB7DE4
:101A300000172BE6BD5A5DB601038A02B7010339D0
:101A4000B6011185012605BD59E420108502260541
:101A5000BD5A0A200785042603BD5A2A39B6010358
:101A60008501274EB6010AB7060B8A01B7010AB6EF
:101A70000108B7060A7F0108B6010FB706098608F4
:101A8000BD603CBD5E9ACE0022BD4C1DBD59188D77
:101A900022CE00AABD4C1DF60609F7010FBD600B52
:101AA000F6060AF70108B6060BB7010ABD591EBDB6
:101AB0005E6B39B6010384FEB7010339B601128AA1
:101AC000FCB70112BD5457261FB60105850F271814
:101AD00084F0B70105B6010684FEB70106B6010A17
:101AE0008A02B7010ABD531839B601128AFC84FB79
:101AF000B70112BD5457267EB6010A8A02B7010A01
:101B0000B601068A01B70106B6010584F08A02B75C
:101B10000105BD53187E545CB601128AFC84F7B7E8
:101B20000112BD5457264FB6010A8A02B7010AB600
:101B300001068A01B70106B6010584F08A01B701E2
:101B400005BD53187E545CB601128AFC84EFB701C0
:101B500012BD54572620B6010584F08A08B7010546
:101B6000B601068A01B70106B6010A84FDB7010A6B
:101B7000BD53187E545C39B601128AFC84DFB7016C
:101B800012BD545726F0B6010584F08A04B701054A
:101B9000B601068A01B70106B6010A84FDB7010A3B
:101BA000BD53187E545CB601128AFC84BFB7011283
:101BB000BD545726C1B6010584F08A02B70105B6A7
:101BC00001068A01B70106B6010A84FDB7010ABD04
:101BD00053187E545CB601128AFC847FB70112BD93
:101BE00054572692B6010584F08A01B70105B60163
:101BF000068A01B70106B6010A84FDB7010ABD5382
:101C0000187E545CB601148A0784FEB70114B6012D
:101C10000684F38A04B70106864C7E28E1B60114D7
:101C20008A0784FBB70114B6010684F38A08B7015A
:101C300006864E7E28E1B601148A0784FDB701149A
:101C4000B6010684F3B70106864D7E28E1B601127F
:101C50008A03B701128601BD60627F010BBD5E6B16
:101C60008649BD28E139B601128A0284FEB7011205
:101C7000864ABD28E1B60111850827037E53CFBDF2
:101C8000545726E17D00172BDCB6010F8A03B701FC
:101C90000FBD5CF3BD5E6B7E5F03B601128A0184EB
:101CA000FDB70112864BBD28E1B601118508270357
:101CB0007E53CFBD545726AD7D00172BA8B6010F1C
:101CC0008A0184FDB7010F20C886017E6062B601DB
:101CD0001284038103260139CE0017BD4C1DB601C5
:101CE0001285012605BD5C7F2003BD5CB3CE0039A3
:101CF0007E4C1DF6010FC48FCA10B601018508265F
:101D00000FC48FCA20B6064485042704C48FCA4076
:101D1000F7010F7E600B966226037E5D684A97622C
:101D2000BD5D7E7E5D409662F60816C50127048182
:101D30000A200281012B037E5D684C9762BD5D7EA7
:101D4000B60C08B101362620D68B270B7A008BC63D
:101D50007ACE5D407E22B08608978BB60136814BE5
:101D600026037E5D167E5D268620978BB60C088145
:101D70004B2705814E270139B701367E5D40860825
:101D80007D00622605BD603C2003BD6062D662CE48
:101D90005D9ABD4C38B70100200B00000104080912
:101DA0000C0A0B0E0F86567D006226028655BD2852
:101DB000E19662260BC690F701154CB70806202065
:101DC0004A260AC6F0F70115F7080620138B0019FA
:101DD00085102604C6D02002C6C0F70115B7080634
:101DE0007E5F03F60111C510262AF60111CA10F70D
:101DF0000111864FBD28E1BD5457270139F6010A6C
:101E0000C4FBF7010ABD5CC9CE0020BD4C1DBD5FFF
:101E10009B7E5CCEF60111C5102608B6010A85042A
:101E2000270139F60111C4EFF70111F6010ACA04BE
:101E3000F7010ABD5E89BD591EBD5F8B8601BD607D
:101E4000628650BD28E1CE08E1BD4C1DBD5FA4BD3A
:101E500034E0BD5E6BB6011285012605BD5C7F20B6
:101E60000785022603BD5CB37E539FBD54572701EF
:101E700039B601128403810326209645857F260901
:101E8000B6011184C081C02711F60104CA04F7010C
:101E900004B6010184FDB7010139F60104C4FBF762
:101EA0000104B601128403810327E6B601018A0208
:101EB000B70101399663B70108203EB601168508BF
:101EC000260139B60817850127148502271CCE0084
:101ED00001BD4C1DB6081743850326E7201BF601FC
:101EE00008C1A0240F7C010820D97D010827057AAC
:101EF000010826CFB6010897638662C601CE0108A5
:101F0000BD28E2B601089763F60112C403C1032697
:101F100007397D00FB2B0139B60108F6010FBD5FC3
:101F200046B1060727122507B10608270B25099693
:101F3000FB8A0497FB7E545CBD5F60E641A600F718
:101F4000010CB7010B39B60108F6010FC5082703CC
:101F50000C20028B6484FC46468140250286403971
:101F6000CE0585FF012616FB0127F7012724037CF8
:101F70000126FE0126FF060C39B601018A04B701CD
:101F80000139B6010184FBB7010139F60111C51011
:101F90002608B6010A84F7B7010A39B6010A8A0889
:101FA000B7010A397D0062262FB601088150242826
:101FB000C682F70108F6010A37CA01F7010A33CED3
:101FC0000200BD4C1DB10108270B7A0108CE0002AA
:101FD000BD4C1D20F0F7010A7E34E0B601018508F2
:101FE000270D7D06432608BD2A308603BD52D5B68F
:101FF000010384FCB70103B6010684FDB701067E28
:00000001FF
